:100000000C947E010C94B6010C94B6010C94B601CC
:100010000C94B6010C94B6010C94B6010C94B60184
:100020000C94B6010C94B6010C949B1E0C946D1F9D
:100030000C947A190C94B6010C94B6010C94B60188
:100040000C94B6010C94B6010C94B6010C94B60154
:100050000C94B6010C94021A0C94B6010C94B601DF
:100060000C94B6010C94B6010C94B6010C94B60134
:100070000C94B6010C94B6010C94B6010C94B60124
:100080000C94B6010C94B6010C94B6010C94B60114
:100090000C94B6010C94B6010C94B6010C94B60104
:1000A0000C94B6010C94B6010C94B6016B046B046D
:1000B00097049704FF041D05350635062805C1057C
:1000C000D205D20584167A168716CF16D316D31604
:1000D000CF16D316D316A816D316B216BC16D3163F
:1000E000D316D316D316CF16D316D316CF16D316D0
:1000F0009516D316D316CC16CC16CC16CC16CC1619
:10010000CC16CC16CC16CC16D116D3168416771670
:10011000D316D316D316D316D316D316D316D31697
:10012000D316D316D116D316D316CF16D316CA1696
:10013000CA16CA16CA16CA16CA16CA16CA16CA16BF
:10014000D116DA1F0120F9200120F9204D2070205E
:10015000F920C720D62053005400550056005F00F8
:100160006000610057005C005D005E0057005900B0
:100170005A005B00580062006200630058000C03E4
:1001800053006F00790075007A00000026036100BB
:1001900069003000330020004400650073006900EE
:1001A00067006E0020005300740075006400690051
:1001B0006F0000000403090409023B00020100A0D3
:1001C000FA090400000103010100092111010001E5
:1001D0002240000705810308000109040100010312
:1001E00000000009211101000122B6000705820369
:1001F000200001120100020000000803A118000104
:10020000000102000105010902A10185020901A105
:1002100000050919012908150025019508750181B6
:10022000020501093009311581257F950275088184
:100230000609381581257F950175088106050C0A88
:1002400038021581257F950175088106C0C005011A
:100250000980A101850319012AB700150126B700FD
:10026000950175108100C0050C0901A101850419D3
:10027000012AA002150126A002950175108100C077
:1002800005010906A1018506050719E029E7150002
:1002900025019508750181020507190029EF150050
:1002A000250195F0750181020508190129059505BB
:1002B00075019102950175039101C005010906A11F
:1002C00001050719E029E715002501950875018149
:1002D000029501750881010507190029FF150026FF
:1002E000FF00950675088100050819012905950587
:1002F00075019102950175039101C00011241FBE83
:10030000CFEFDAE0DEBFCDBF04B603FE18C08091A8
:100310008B0290918C02A0918D02B0918E02873059
:10032000904BA740B04B59F410928B0210928C0264
:1003300010928D0210928E02E0E0F8E3099511E030
:10034000A0E0B1E0E8E5F3E402C005900D92A43826
:10035000B107D9F722E0A4E8B1E001C01D92AB38A3
:10036000B207E1F70E94F4110C94AA210C9400004A
:1003700081E0089581E008950C94BA0108950C94E9
:10038000BE011F93CF93DF9300D000D01F92CDB753
:10039000DEB749835A836B833091870189819A81C3
:1003A000311114C0662359F0222349F00E947008CD
:1003B000182F682F89819A810E941B0803C00E9410
:1003C0004508182F69817A81812F04C00E94700826
:1003D00069817A810F900F900F900F900F90DF91AD
:1003E000CF911F910C948B0FFC01262F40815181DE
:1003F0006281738184810C94C10181E00895CF935F
:10040000DF93EC0160E00E94F401BE01DF91CF9127
:100410000C94BF010C94B8100C94B41008950E9471
:10042000C5060E940E022FEF84E39CE0215080401D
:100430009040E1F700C000000C94281A0F931F931E
:10044000CF93DF938C0161E00E94F401EC01B801CD
:100450000E94BC018823F1F1B801CE010E94C617A9
:100460008823C1F1B801CE010E948A14882391F13A
:10047000B801CE010E942217882361F1F801828120
:10048000882309F1CB358DE5D807C1F050F4C115AB
:10049000FCE5DF0781F0CF3DDC45A9F40E94A10D0A
:1004A00019C0CC35EDE5DE0761F0CD35DD4559F4F9
:1004B0000E94EA0C08C00E940F020CC00E94F30CBC
:1004C00002C00E94F60CC801DF91CF911F910F91DD
:1004D0000C94B80180E0DF91CF911F910F910895A6
:1004E0000E945D190C9489020E948C020C9463197D
:1004F00008950C94780281E008950C947B0208958D
:10050000CF93C82F0E9479028C2F0E947D02CF9139
:10051000089580E00C9480020E9422180C948002BE
:100520000E94221890918601891721F080938601FC
:100530000C9480020895CF93DF93CDB7DEB72B974D
:100540000FB6F894DEBF0FBECDBF4F8358876987C3
:100550007A878B8761110E94360C9E012F5F3F4F77
:1005600086E0F90111928A95E9F785E0FE01379658
:10057000D90101900D928A95E1F789819A814C8188
:100580005D81452B31F09F3F31F491E08F3F19F4AD
:1005900003C091E001C090E090FF09C049815A81F9
:1005A0006B817C818D819E810E94570B05C0C901A2
:1005B0000E94FD018111F2CF2B960FB6F894DEBF99
:1005C0000FBECDBFDF91CF910895FC018081918155
:1005D0000E94B2080895CF93882309F4A9C0C82FB8
:1005E0008238C1F40E94221881FDA2C069E3809183
:1005F0000201909103010E9418190E94580C2FEFDC
:1006000081EE94E0215080409040E1F700C000006E
:1006100069E319C0833801F50E94221880FD88C063
:1006200063E580910201909103010E9418190E94D4
:10063000580C2FEF81EE94E0215080409040E1F77C
:1006400000C0000063E580910201909103010E94C7
:100650002319CF910C94580C8438C1F40E942218AD
:1006600082FD66C067E480910201909103010E94BF
:1006700018190E94580C2FEF81EE94E02150804011
:100680009040E1F700C0000067E4DDCF8CEF8C0FF5
:10069000813AF8F48C2F0E94D916811149C06C2F31
:1006A00080910201909103010E949818882349F0DB
:1006B0006C2F80910201909103010E9423190E94E6
:1006C000580C6C2F80910201909103010E9418191F
:1006D000C0CF80E28C0F883048F4C77081E001C041
:1006E000880FCA95EAF70E94190CB3CFEBE5EC0F1F
:1006F000E33040F4F0E0E95BFE4F808190E0CF9181
:100700000C945618E8E5EC0FE73150F4F0E0EE0FEA
:10071000FF1FE75EFE4F80819181CF910C946C1892
:10072000CD3E30F08C2F0E947912CF910C944B1358
:10073000CF910895882309F464C0823879F40E9427
:10074000221881FF5EC069E380910201909103014C
:100750000E9418190E94580C69E310C08338B1F444
:100760000E94221880FF4DC063E5809102019091A4
:1007700003010E9418190E94580C63E58091020140
:10078000909103010E9423190C94580C843879F439
:100790000E94221882FF35C067E480910201909187
:1007A00003010E9418190E94580C67E4E7CF9CEFE0
:1007B000980F913A10F4682FE1CF90E2980F98309B
:1007C00050F4877091E001C0990F8A95EAF7892F5C
:1007D0000E941F0CD9CF9BE5980F933020F480E046
:1007E00090E00C94561898E5980F973120F480E02B
:1007F00090E00C946C188D3E20F00E94D4120C9462
:100800004B1308951F93CF93DF93182FEB010E9492
:10081000EB02209741F08FE99FE00197F1F700C0CC
:1008200000002197F6CF812FDF91CF911F910C947B
:100830009A03893319F060E070E002C060E570E06F
:100840000C940204882321F00E94190C0C94580C7B
:100850000895882321F00E941F0C0C94580C0895D1
:10086000CF92DF92EF92FF920F931F93CF93DF937C
:100870007C01D62FC72FFC011281058102950F70D4
:100880000E940F0C8823B9F01123A9F08C2F807FD0
:10089000803421F080E28D0F883068F080916F0203
:1008A00082FD09C082E00E94B80C0E940F0C91E00A
:1008B000D82ED92601C0D12CCC2EC2948FE0C822CC
:1008C0008C2D90E08C30910508F0CFC1FC01EA5AE4
:1008D000FF4F0C9441218C2F807FCF70882311F023
:1008E000C295C07F112399F0CC2309F4AAC180E2FC
:1008F0008D0F883010F0D11104C08C2F0E94190C7C
:1009000003C08C2F0E94290C0E94580C9AC18D2F75
:100910000E949A03CC2309F4A8C180E28D0F88308D
:1009200038F1DD2329F18C2F0E942F0C24C08C2F4D
:10093000807FCF70803211F0C295C07FDD2319F027
:10094000D130A1F13DC080916F0282FF17C0112309
:1009500049F0CC2329F08C2F0E94190C0E94580CCE
:1009600080E070C180E00E949A03CC2309F47DC12D
:100970008C2F0E941F0C0E94580C77C1112371F01C
:10098000002341F0013031F40E94390C8C2B0E947D
:10099000410C6BC10E94390C8C2B1DC0002319F037
:1009A000013009F462C10E944E0C25C0112321F0D0
:1009B000063008F05AC10EC0053008F056C11BC001
:1009C000112361F0002331F0F701858180FF39C1E7
:1009D0008F7085838C2F0E94220447C1002359F019
:1009E000D93309F03FC1FFEF07EE13E0F1500040AB
:1009F0001040E1F735C18C2F0E94290436C18C2F9D
:100A000086958695837019F0813061F02EC111238F
:100A100021F08D2F9C2F937002C080E090E00E9407
:100A200056182BC1112321F08D2F9C2F937002C0DB
:100A300080E090E00E946C1820C18D2F112319F0E6
:100A40000E94791202C00E94D4120E944B1315C159
:100A50008C2F837009F047C011110BC12D2F2295E7
:100A600026952770220F220F6D2F6F70862F90E032
:100A7000A0E0B0E0022E04C0880F991FAA1FBB1F80
:100A80000A94D2F7D4FF10C04FE050E060E070E06D
:100A900004C0440F551F661F771F2A95D2F7409553
:100AA00050956095709503C040E050E0BA01C6953E
:100AB000C695C3708A019B01082B192B2A2B3B2B4F
:100AC000C901B801C23049F058F4C13019F00E9490
:100AD0003107CFC00E941F07CCC00E944307C9C086
:100AE0000E941D07C6C0112319F08C2F817001C010
:100AF0008695882309F4BDC02D2F22952695277051
:100B0000220F220F6D2F6F70862F90E0A0E0B0E0D3
:100B1000022E04C0880F991FAA1FBB1F0A94D2F788
:100B2000D4FF10C04FE050E060E070E004C0440F1C
:100B3000551F661F771F2A95D2F7409550956095EF
:100B4000709503C040E050E0BA01C695C695C370E9
:100B50008A019B01082B192B2A2B3B2BC901B801B9
:100B6000C23049F058F4C13019F00E94F60781C034
:100B70000E94E4077EC00E9408087BC00E945707BD
:100B800078C0CF70112339F08C2F0E947D078D2FF4
:100B90000E9422046EC08D2F0E9429048C2F0E9477
:100BA0009E0767C0D23F21F128F4D03F41F0D13FEA
:100BB000C1F043C0D33F19F1D43F79F03EC01123B7
:100BC00041F0053008F051C08C2F8F710E94C3078F
:100BD0004CC0063008F049C0F7CF80916F0282FF09
:100BE00018C0112339F08C2F8F710E947D073DC0F2
:100BF0001123C9F38C2F8F710E949E0736C01123D9
:100C000029F08C2F8F710E9468072FC00E94630704
:100C10002CC0112349F0CF718C2F0E947D0763E017
:100C20008C2F0E949D0C21C081E00E94B80C0230E4
:100C3000E0F082E00E94B80C18C0112331F00023CC
:100C400091F28D2F0E94EB0210C0002399F2D9334C
:100C500049F41FEF27EE33E0115020403040E1F718
:100C600000C000008D2F0E949A0388EF8C0D843005
:100C700020F40E9422180E948002DD20C9F00E9408
:100C80000B0C80FD15C0F70112820E94050C0E941A
:100C90007D07C7010E9479060E94050CDF91CF9164
:100CA0001F910F91FF90EF90DF90CF900C949E07D3
:100CB000DF91CF911F910F91FF90EF90DF90CF9038
:100CC00008950F931F93CF93DF93EC01688179818F
:100CD0008A810E94BD088C010E941A080E940B079D
:100CE000B801CE010E943004DF91CF911F910F9186
:100CF0000895CF93DF93EC01988189812B813C810A
:100D0000232B31F08F3F31F481E09F3F19F403C072
:100D100081E001C080E080FD1DC0CE010E941E0266
:100D2000811110C00E940F0C8823A1F08A818823B2
:100D300089F080916F0282FD0DC082E0DF91CF913A
:100D40000C94B80CCE010E946106CE01DF91CF91C8
:100D50000C94FF01DF91CF91089580E090E00E9414
:100D6000561880E090E00E946C180E94360C0E9499
:100D7000580C0E947C140C944B13809102019091AA
:100D800003010E942E190C94AD060E94260C0C94AF
:100D9000BD0692959F70963079F010F4925001C084
:100DA0009A50923068F4803F69F018F4883E40F41D
:100DB00009C0843F29F406C0883E20F0813F11F02D
:100DC00080E0089581E00895FC01808191810E9476
:100DD000B2080E94C9060895CF93DF9300D000D0D7
:100DE0001F92CDB7DEB70F900F900F900F900F901E
:100DF000DF91CF910895CF93DF9300D000D000D042
:100E0000CDB7DEB726960FB6F894DEBF0FBECDBFC6
:100E1000DF91CF910895089508950C940C070C94D8
:100E20000D070E940F0760939B0170939C018093B4
:100E30009D0190939E010C94AD060C9411070F93A5
:100E40001F9300919B0110919C0120919D01309175
:100E50009E01602B712B822B932B1F910F910C9471
:100E600011070F931F9300919B0110919C012091FA
:100E70009D0130919E0160237123822393231F9152
:100E80000F910C9411070F931F9300919B011091E8
:100E90009C0120919D0130919E016027712782273E
:100EA00093271F910F910C9411070C940C070E942B
:100EB00055076093970170939801809399019093DF
:100EC0009A010C94AD0660E070E0CB010C945707DA
:100ED0000F931F9341E050E060E070E08A019B01B6
:100EE00004C0000F111F221F331F8A95D2F7C901BA
:100EF000B8011F910F910C9457070F931F9341E076
:100F000050E060E070E004C0440F551F661F771F7B
:100F10008A95D2F78091970190919801A0919901BB
:100F2000B0919A018A019B01082B192B2A2B3B2B8C
:100F3000C901B8011F910F910C9457070F931F938C
:100F400041E050E060E070E004C0440F551F661FB0
:100F5000771F8A95D2F7409550956095709580914E
:100F6000970190919801A0919901B0919A018A01FD
:100F70009B01082319232A233B23C901B8011F9190
:100F80000F910C9457070F931F9341E050E060E0DE
:100F900070E004C0440F551F661F771F8A95D2F773
:100FA0008091970190919801A0919901B0919A0137
:100FB0008A019B01082719272A273B27C901B80165
:100FC0001F910F910C9457070F931F930091970156
:100FD000109198012091990130919A01602B712B09
:100FE000822B932B1F910F910C9457070F931F93F4
:100FF00000919701109198012091990130919A01E7
:1010000060237123822393231F910F910C94570720
:101010000F931F93009197011091980120919901CE
:1010200030919A0160277127822793271F910F9192
:101030000C9457070895990F990F890FE82FE6959B
:10104000E695E695877051E001C0550F8A95EAF75D
:1010500085E0E89FF0011124E857FE4F20E030E0E2
:1010600070E04081CB01022E02C0969587950A94CC
:10107000E2F78170819584278523842781932F5FF0
:101080003F4F2530310569F70895990F990F890F62
:10109000682F669566956695982F977085E0689F8E
:1010A000B001112440E050E080E0FB01E40FF51FA7
:1010B000E857FE4F208130E0092E02C03695279573
:1010C0000A94E2F721703327042E01C0220F0A94FC
:1010D000EAF7822B4F5F5F4F4530510531F7089596
:1010E000BF92CF92DF92EF92FF920F931F93CF9315
:1010F000DF938C01C0909701D0909801E090990106
:10110000F0909A0180919B0190919C01A0919D018A
:10111000B0919E01C82AD92AEA2AFB2ACFE1D0E061
:10112000D701C6010C2E04C0B695A7959795879553
:101130000A94D2F780FD04C0219790F7B12C07C024
:10114000BC2EB8018C2F0E949F0F0197A9F38B2D05
:10115000DF91CF911F910F91FF90EF90DF90CF9093
:10116000BF900895CF93DF93EC010E947008BE01F9
:101170000E949F0FDF91CF9108951F93CF93DF932C
:10118000EB0190918701992321F0CB010E94B208D5
:1011900013C0882349F0CB010E947008182F682FD4
:1011A000CE010E941B0804C0CB010E944508182FE5
:1011B000BE01812F0E949F0FDF91CF911F91089553
:1011C0001F93CF93DF93C0919F0116E08091A00100
:1011D000C81799F0D0E01C9FF0011D9FF00D11245D
:1011E000EF55FE4F408151816281738184819581E9
:1011F0000E94FB062196C770E9CFDF91CF911F9126
:1012000008954091D1015091D2016091D301709124
:10121000D4018091D5019091D6010C94FB06EF92F8
:10122000FF920F931F93CF93DF938091D601829506
:101230008F7009F065C08091D301882309F460C0E4
:1012400080919F01F090A0011091D1010091D201F5
:101250006091D4017091D50191E01F3F09F090E0B9
:10126000C0910001D0910101292F96E0E92E8F1540
:1012700009F446C06115710521F00F3F21F030E0FF
:1012800003C031E001C0322F90E030FD36C0E89E4F
:10129000F001E99EF00D1124DF01AF55BE4F11960C
:1012A0003C911197301329C03C91311326C01296FE
:1012B0003C911297311121C013964D915C91149776
:1012C000461B570B4C175D07C0F48091D6018F70F9
:1012D00080618093D601EA55FE4F80818F708061D6
:1012E000808381ED91E00E947906DF91CF911F917B
:1012F0000F91FF90EF900C94E00801968770B7CFA4
:10130000DF91CF911F910F91FF90EF9008959F92E1
:10131000AF92BF92CF92DF92EF92FF920F931F9303
:10132000CF93DF93CDB7DEB761970FB6F894DEBFEA
:101330000FBECDBF8C0185E0F801DE011D96019046
:101340000D928A95E1F7D8011296EC909091D10117
:10135000E091D2012091D4013091D50121153105C0
:1013600031F0EF3F31F481E09F3F19F403C081E099
:1013700001C080E0B82FB1709B2E80FD47C1D8011D
:101380004C9111965C9111971396AD90BC90149767
:1013900081EDC82E81E0D82EF090D301B501621BFB
:1013A000730B2091000130910101FF2009F4D9C095
:1013B0008091D6016217730708F095C0282F207F0F
:1013C00009F052C05E1313C0491311C0FE2CE11086
:1013D0000EC08F7080618093D6010E940109C60102
:1013E0000E9479068091D601F80185834DC1AB2812
:1013F00031F05F3F31F481E04F3F19F403C081E0E9
:1014000001C080E080FD03C081E08E2502C080E045
:1014100090E0F82FF170FF2E80FF1CC080919F019B
:101420002091A00136E0821709F40BC190E0389FAB
:10143000F001399FF00D1124EF55FE4F61815613D5
:1014400006C06081461303C06281E61203C00196A4
:101450008770E9CFFE2CEE2009F416C18091D601E9
:1014600081608093D60154C05E1306C0491304C046
:10147000E11002C0F80199C0C8010E94E406882367
:1014800061F1EE2051F12091D601822F82958F706B
:1014900090E0029774F08091D1019091D2019887E9
:1014A0008F831986BB86AA862C87CE0107960E9459
:1014B000790686E0F801A1EDB1E001900D928A95E0
:1014C000E1F70E940F090E9401090AC05E1711F19D
:1014D000C8010E94E40681112CC0C8010E9479064F
:1014E000FF24F394D1C0282F207F81F77A2DB98A69
:1014F000A88A6E2D89890E94EC0681ED91E00E94F8
:10150000790686E0D6011D928A95E9F70E940109C5
:10151000F12CBAC04913DCCFE110DACFF801858392
:10152000C8010E94790686E0D6011D928A95E9F7E6
:10153000ABC0EE2091F22091D601822F82958F7060
:1015400090E002970CF4B5CF8091D1019091D20137
:101550009A8389831B82BD82AC822E83CE01019641
:10156000A6CF6217730708F044C0FE2CEE2009F4E2
:10157000B4CF5E1330C049132EC02091D60120FD98
:1015800021C0822F82958F70482F50E04115510560
:10159000C9F0F80125834F30510541F08F5F982F36
:1015A0009295907F822F8F70892B8583C8010E942E
:1015B000790686E0F801A1EDB1E001900D928A95DF
:1015C000E1F73CC086E0F801A1EDB1E001900D9299
:1015D0008A95E1F759C0C8010E94E406811169CFDC
:1015E0008091D60181608093D601C8010E9479065E
:1015F0004BC07A2DB98AA88A6E2D89890E94EC0683
:1016000086E0D6011D928A95E9F718C0EE2009F40C
:1016100064CFC8010E94E406F82E882309F45DCF48
:1016200086E0F801A1EDB1E001900D928A95E1F715
:1016300081ED91E00E94E5020E940F090E940109DC
:1016400023C04D875E878D859E850E94B208292F15
:1016500022952F70223028F49F7039F0811105C037
:101660000BC0243028F49F7049F4805E883020F04D
:10167000C8010E9479069F2CF92C06C0D801159646
:101680009C91907F91F7F8CF8F2D61960FB6F894CB
:10169000DEBF0FBECDBFDF91CF911F910F91FF90A5
:1016A000EF90DF90CF90BF90AF909F9008951F93E1
:1016B000CF93DF93CDB7DEB72C970FB6F894DEBF8C
:1016C0000FBECDBF4F83588769877A878B879C87EA
:1016D000CE0107960E9487098823D1F09F818885D3
:1016E0002A853B85232B31F08F3F31F481E09F3FEA
:1016F00019F403C081E001C080E080FD47C04F8144
:10170000588569857A858B859C850E94FB063EC03D
:1017100086E0FE013796DE01119601900D928A95C2
:10172000E1F7FF81E8856A857B856115710531F0F8
:10173000EF3F31F481E0FF3F19F403C081E001C0C5
:1017400080E080FD23C02091A00130E0C901019616
:101750008770992740919F0150E084179507F1F118
:10176000F983EA837D836C8396E0929FD001939FF7
:10177000B00D1124AF55BE4FFE01319601900D9270
:101780009A95E1F78093A0010E94E00816E080910D
:101790009F019091A001891771F1189FC001112438
:1017A0008F559E4F0E948709882329F1E0919F0160
:1017B0001E9FF0011124EF55FE4F4081518162813F
:1017C0007381848195810E94FB0680919F0190E046
:1017D00001968770992780939F01D9CF0E94C506F3
:1017E0001092A00110929F01E1EDF1E086E0DF018F
:1017F0001D928A95E9F72C960FB6F894DEBF0FBEBE
:10180000CDBFDF91CF911F9108958091F70185950C
:101810008595859508958091F70187700895909139
:10182000F701977081E009F480E0089580911A0231
:10183000089590911A02892B80931A020895809539
:1018400090911A02892380931A02089510921A0225
:10185000089590911902892B80931902089580951B
:101860009091190289238093190208951092190208
:1018700008958091F801089508950C943C0C0C94FF
:101880003D0C90916F0292FD08C09091F80198175D
:1018900021F08093F8010C943F0C08958091F80199
:1018A000882329F01092F80180E00C943F0C0895F1
:1018B000CF93DF93E0910201F091030180911A022E
:1018C0008083E0910201F0910301908180911902DF
:1018D000892B80838091F801882381F0E0910201B7
:1018E000F09103019081892B808380910201909176
:1018F00003010E94821881110E944E0CC0910201C6
:10190000D091030140E250E067ED71E0CE010E940A
:101910005B21892B69F080E2FE01A7EDB1E0019027
:101920000D928A95E1F7CE01DF91CF910C942E189C
:10193000DF91CF9108950C943C0C90916F0292FD31
:1019400010C098E0899F90011124262B2093F70165
:101950000E947D078091F7018595859585950C946A
:101960009B0C0C947D071092F70180E00C949B0C6B
:101970002091F701809582238093F701982F97702B
:1019800099F430E0482F082E000C550B241735072A
:1019900059F090916F0292FD07C0859585958595C8
:1019A0000E949E070C94B30C089590916F0292FBD5
:1019B000222720F9281769F080FB92F990936F0293
:1019C00080916E0290916F020E941D0D82E00C9436
:1019D000B80C089580916F0282FB882780F991E00E
:1019E00089270C94D50C81E00C94D50C80E00C94E4
:1019F000D50C80E090E00E94702121E0893E9E4F4E
:101A000009F020E0822F089582E090E00C94682194
:101A100083E090E00C946821CF9384E090E00E94F2
:101A20006821C82F82E290E00E9468212C2F30E0CC
:101A3000A901582BCA01CF910895CF93C92F682FC0
:101A400084E090E00E9476216C2F82E290E0CF91BA
:101A50000C947621AB01BC018FE090E00C948821BE
:101A6000AB01BC0183E190E00C94882160E070E060
:101A7000CB010C94300D60E070E0CB010E942A0D88
:101A80000C94360D69EE7EEF80E090E00E94942188
:101A900060E082E090E00E94762160E083E090E0E8
:101AA0000E94762110929B0110929C0110929D0140
:101AB00010929E0160E084E090E00E94762160E058
:101AC00082E290E00E94762160E085E090E00E9452
:101AD000762160E086E090E00E9476216FEF87E05B
:101AE00090E00E94762140E050E0BA0188E090E06A
:101AF0000E94882160E08DE090E00E94762140E025
:101B000050E0BA0188E190E00E94882160E087E11E
:101B100090E00E94762140E050E0BA018CE190E034
:101B20000E94882160E070E080E290E00E949421B1
:101B300040E050E0BA0188E190E00E9488210C94D6
:101B40003B0D0C94420D682F8EE090E00C947621B2
:101B50000E94E71960932402709325028093260265
:101B600090932702609320027093210280932202B7
:101B700090932302089585B7806885BF85B78068F4
:101B800085BF089581E008950C94C20D08950C94CA
:101B9000C60D0C94C60D0C94C90D0C94C60D0C9476
:101BA000CD0D0C94C60D0E94BB0D8BE790E10E94F9
:101BB00018180E94D10D0C94CF0D0E94C70D0C94E3
:101BC000C60D0E947E100C947F020E94D2190E94C2
:101BD00055110E94E10D0C94CB0D8F929F92AF9204
:101BE000BF92CF92DF92EF92FF920F931F93CF930A
:101BF000DF93CDB7DEB72A970FB6F894DEBF0FBEDE
:101C0000CDBF0E946A11982E81110E94A80D8BE110
:101C1000A82E82E0B82E00E010E0802E802F0E94D7
:101C2000A210D82EF501C1905F01C826B1F40F5F54
:101C30001F4F0530110589F78FEF89838A831B8237
:101C40000E94DB198160782F9D838C8349815A81A2
:101C50006B818D810E949B022FC08091280281FDA3
:101C60000E94A810E12CFF24F3948C2D8F21F1F019
:101C70000E94C40D882399F0EE828F82DF2081E0DC
:101C800009F480E088870E94DB198160782F9A87A9
:101C900089874E815F8168858A850E949B02F80151
:101CA000E55EFD4F8081F826F08206C0E394FF0CCC
:101CB000F4E0EF12DACFBBCF81E0911001C080E0F9
:101CC0002A960FB6F894DEBF0FBECDBFDF91CF913D
:101CD0001F910F91FF90EF90DF90CF90BF90AF904A
:101CE0009F908F9008950E94ED0D0E9469130C94AF
:101CF0009002CF93DF930E94A40FEC01811521E5A0
:101D0000920708F045C0811530E5930708F094C0AC
:101D1000883E910528F5803E910508F0F8C0883A84
:101D2000910570F4853A910508F07CC081309105E9
:101D300009F475C008F4E8C0049708F0E8C0E4C0EE
:101D40008F3B910508F0E0C0C85AD0E0CC0FDD1FF2
:101D5000C65BDE4F0990D881C02DCE019464D8C0F7
:101D6000811540E2940758F4811551E0950708F079
:101D7000CEC08D3E910508F4C7C09065C9C0C1159D
:101D800080E4D80708F4C0C0DF70CE01906AC0C0FC
:101D9000811525E59207A8F4811534E5930708F02D
:101DA00095C0811543E5940708F07BC0811552E585
:101DB000950708F061C0D82FCC27CE01816F906ABB
:101DC000A7C0C11589E5D807A0F4C11528E5D20739
:101DD00008F082C0C11536E5D30708F095C08C2FF6
:101DE0000E9438108F7190E0D82FCC27CE019062DE
:101DF0008FC0C1154AE5D40708F474C0CE019056CF
:101E00008115904208F080C08D2F8F710E9438108C
:101E1000DD27D0628F71AE01582BCA0179C081E0F5
:101E200090E076C0C55AD0E0C858DE4F8881C82FF0
:101E3000D0E0CE0190646CC074E0969587957A9559
:101E4000E1F7282F23703C2F337081E090E002C02F
:101E5000880F991F3A95E2F79C68AC01522B9A01C2
:101E60009C2F9F709695969550E2959FE0011124C6
:101E7000C9018C2B9D2B4CC08370992721E030E049
:101E800002C0220F331F8A95E2F79C2F96959695F4
:101E900080E2989FE0011124C22BD32BCE019C68D5
:101EA00037C08370992721E030E002C0220F331F32
:101EB0008A95E2F79C2F9695969540E2949FE001D3
:101EC0001124C22BD32BCE019A6822C0D82FCC2745
:101ED000CE01846F906A1CC0DC2FCC27CE01806FAE
:101EE000906A16C08C2F8F700E94381094E0D6959F
:101EF000C7959A95E1F7CF70D0E0DC2FCC27D06959
:101F00009E01282BC90104C080E090E001C0CE01F1
:101F1000DF91CF910895E72FF0E095E0899FE00DE4
:101F2000F11D1124EE0FFF1FEE0FFF1FE60FF11D35
:101F3000EE0FFF1FEA5AFE4F8591949108950E947B
:101F40008B0F0E94790E08958238910569F1B0F4E3
:101F50008133910509F46DC048F48932910509F483
:101F600063C08A32910509F469C0089585339105EB
:101F700009F455C089339105B9F00895833E910560
:101F800069F138F4803E9105B1F0823E910509F186
:101F90000895863E9105A9F1873E9105B9F1843EE9
:101FA000910509F064C023C020916E0220FD4FC04E
:101FB00021FD4DC0089580916E0280FD44C0809146
:101FC0006F0280FF44C080916E0284FD42C083EEA8
:101FD0004DC080916E0282FF38C0F5CF80916E02B5
:101FE00082FD33C080916F0280FD31C0ECCF8091C3
:101FF0006F0281FF32C080916E0284FD2AC087EE9D
:1020000035C080916E0283FF26C0F5CF80916E02AD
:1020100083FD21C080916F0281FD1FC0ECCF8091B4
:102020006E0285FD1CC01DC080916E0285FD19C029
:1020300016C080916E0286FD16C017C080916E0298
:1020400086FD13C010C089E311C082EE0FC080EE80
:102050000DC080E00BC086EE09C084EE07C089E2A7
:1020600005C085E303C08AE201C081E390E00895E2
:1020700090916E0292FF0DC0282F2871283019F41C
:10208000877F846006C0282F2471243011F48B7F51
:10209000886093FF0DC0282F2871283119F4877E9E
:1020A000846106C0282F2471243111F48B7E88614D
:1020B00020916F0220FF0DC0382F3871383019F48D
:1020C000877F816006C0382F3171313011F48E7FE7
:1020D000886021FF0DC0282F2871283119F4877ED0
:1020E000816106C0282F2171213111F48E7E886113
:1020F00094FD877E089580E0089508950E94F90C6C
:10210000811102C00E94A10D0E94040D809328023B
:102110000E940C0D90936F0280936E020E947D10BE
:102120000E94080D682F70E080E090E00E941D077B
:1021300060919701709198018091990190919A0115
:102140000C945507E82FF0E0EB58FD4F808108957F
:10215000089580EA8A95F1F7089500C008950C94D7
:10216000A91008950C94B1100C94B2100C94B110F5
:102170000C94B610F894E82FE295EF70F0E031A1DE
:10218000282F2F7081E090E001C0880F2A95EAF790
:10219000982F9095932391A392A1892B82A3789451
:1021A00008950F931F93CF93DF93CFE7D1E08991E9
:1021B0008F3F11F00E94BA1081E0C438D807B9F7F8
:1021C000CBE7D1E00FE711E089918F3F11F00E943A
:1021D000BA100C171D07C1F7DF91CF911F910F9116
:1021E0000895CF92DF92EF92FF920F931F93CF93B8
:1021F000DF938C01C62FD0E0CE0181589E4F7C0129
:10220000FC0190819F3F09F447C0D62EF894E92F36
:10221000E295EF70F0E081A19F7021E030E001C015
:10222000220F9A95EAF7822B81A382A12095282379
:1022300022A378940E94AD10EBE7F1E04FE751E064
:1022400031E0C12C21912F3F89F0A22FA295AF70D0
:10225000B0E090968C9190E02F7002C09595879594
:102260002A95E2F780FD02C0832F01C080E0C82AD2
:10227000330F4E175F0731F7F70180818F3F11F061
:102280000E94BA1061E0C11001C060E08D2D0E9473
:10229000AF10C00FD11FC882DF91CF911F910F9156
:1022A000FF90EF90DF90CF9008950E94D11085E0CD
:1022B000E5E7F2E0DF01982F1D929A95E9F7E0E754
:1022C000F2E0DF011D928A95E9F785E00E94B111E5
:1022D0000C940A02FF920F931F93CF93DF9300D0C9
:1022E00000D01F92CDB7DEB78E010F5F1F4F85E084
:1022F000F80111928A95E9F7F12C6F2DC8010E941F
:10230000F110F394F5E0FF12F8CF45E050E0B8018A
:1023100080E792E00E945B21FF24F394009709F488
:10232000F12C892B41F085E0F801A0E7B2E00190A3
:102330000D928A95E1F72F2D45E065E772E080E781
:1023400092E00E94B2110E940C028F2D0F900F900C
:102350000F900F900F90DF91CF911F910F91FF90F1
:1023600008950895FF920F931F93CF93DF938C01ED
:10237000F62ED72FC42F222349F081E080932B0221
:102380000E94DB1990932A028093290280912B02EC
:102390008823C1F08091290290912A020E94F319AA
:1023A000059780F0EF2DFD2FD8014C2F50E0CD0187
:1023B000801B910B841795071CF48D918193F7CFA7
:1023C00010922B02DF91CF911F910F91FF900895F2
:1023D0000E94F31B0E94E50D0C94FF1B0E94031C3E
:1023E0000E94730E0C941D1C0E9479190E94DA1B26
:1023F0000E94D30D0E94E8110E94EE110E94DD0D93
:10240000FBCF8091320280FF06C06091090170E02D
:10241000660F771F26C081FF04C06091090184E028
:1024200005C082FF07C06091090188E0689FB00184
:10243000112417C0909131029923D1F060910801C5
:10244000961788F72091090188E0289F90011124B0
:10245000929FA001939F500D112470E0CA010E9429
:102460002D216038710540F46115710519F406C01D
:1024700068E070E0862F08958FE7089581E0089561
:102480008091320280FF08C06091050170E075956F
:1024900067957595679521C081FF06C0609105011C
:1024A00070E07595679519C082FF04C060910501C1
:1024B00070E010C090913002992399F0609104016E
:1024C0009617A0F780910501899FC001112470E043
:1024D0000E942D216038710540F46115710519F4D1
:1024E00006C061E070E0862F08958FE7089581E0CF
:1024F00008958D3E21F40E940112819504C08E3E04
:1025000029F40E9401128093360208958F3E21F42F
:102510000E940112819504C0803F29F40E9401129B
:10252000809335020895893F19F40E94401205C036
:102530008A3F31F40E9440128195809337020895BA
:102540008B3F21F40E944012819504C08C3F29F4F6
:102550000E9440128093380208959FE0980F9830AF
:1025600078F421E030E0A90102C0440F551F9A958C
:10257000E2F7CA0190913402892B809334020895C6
:102580008D3F21F48091320281600BC08E3F21F497
:1025900080913202826005C08F3F29F4809132021F
:1025A00084608093320208958D3E39F49091360212
:1025B00097FF35C01092360259C08E3E29F4909193
:1025C00036021916BCF32BC0909135028F3E29F4C8
:1025D00097FF25C01092350249C0803F19F41916A3
:1025E000CCF31DC090913702893F29F41916BCF431
:1025F000109237023BC08A3F19F497FF10C0F8CF02
:102600008B3F39F49091380297FF09C0109238023D
:102610002DC08C3F21F4909138021916BCF39FE035
:10262000980F983080F421E030E0A90102C0440FF7
:10263000551F9A95E2F7CA0180959091340289233B
:102640008093340213C08D3F21F4809132028E7F3B
:102650000BC08E3F21F4809132028D7F05C08F3FE9
:1026600029F4809132028B7F80933202809135026F
:10267000811106C080913602811102C01092310290
:1026800080913702811106C080913802811102C009
:102690001092300208950E94DB1920913502211119
:1026A00004C020913602222321F090932F028093C0
:1026B0002E0220913702211104C0209138022223DA
:1026C00021F090932D0280932C0283E392E00C94EE
:1026D0004818EF92FF920F931F93CF93DF9300D090
:1026E00000D000D0CDB7DEB786E0E3E3F2E0DE0154
:1026F000119601900D928A95E1F7E0903502F090E5
:102700003602009137021091380210923502109271
:1027100036021092370210923802E11003C0FF20F7
:1027200009F45DC080912E0290912F020E94F3194E
:10273000AC0190913102992339F020910A0130E0E7
:102740002417350758F04BC020910B018AE0289FD1
:10275000900111242417350718F041C09F3F19F04C
:102760009F5F90933102EE2061F00E9401121E14CF
:1027700014F09FEF01C091E0989F902D1124909349
:102780003502FF2061F00E9401121F1414F09FEF28
:1027900001C091E0989F902D1124909336023091C2
:1027A00035023323E1F0209136022223C1F045EBBC
:1027B0003403C0011124992319F09093350203C00A
:1027C00081E08093350235EB2303C0011124992366
:1027D00019F09093360203C081E080933602011114
:1027E00003C0112309F45DC080912C0290912D0249
:1027F0000E94F319AC0190913002992339F0209195
:10280000060130E02417350758F04BC0209107012E
:102810008AE0289F900111242417350718F041C041
:102820009F3F19F09F5F90933002002361F00E9458
:102830004012101614F09FEF01C091E0989F902D68
:10284000112490933702112361F00E944012111657
:1028500014F09FEF01C091E0989F902D1124909368
:102860003802309137023323E1F0209138022223DD
:10287000C1F045EB3403C0011124992319F0909362
:10288000370203C081E08093370235EB2303C00198
:102890001124992319F09093380203C081E08093AA
:1028A00038028091350281110BC08091360281116E
:1028B00007C080913702811103C0809138028111D5
:1028C0000E944B13EB82FC820D831E8386E0FE0187
:1028D0003196A3E3B2E001900D928A95E1F7269636
:1028E0000FB6F894DEBF0FBECDBFDF91CF911F9121
:1028F0000F91FF90EF900895E3E3F2E086E0DF01AF
:102900001D928A95E9F710923102109230021092CE
:1029100032020895CF93DF93EC01FB01828188237B
:1029200009F43CC1C430FDE5DF0760F4CB3F9CE512
:10293000D90788F49E0122503C452431310508F026
:102940002EC109C0C236EDE5DE0729F0C63AFDE525
:10295000DF0709F024C10E940C0D90936F02809351
:102960006E02C1318CE5D80709F4C6C008F042C038
:10297000C930ECE5DE0709F49BC000F5C5308CE5F5
:10298000D80709F485C078F4C330ECE5DE0709F414
:1029900078C008F07AC0C230DC4509F0F5C08091FB
:1029A0006E028160EFC0C7309CE5D90709F478C09A
:1029B00008F07AC080916E028061E4C0CD30FCE501
:1029C000DF0709F487C058F4CB309CE5D90709F438
:1029D00079C008F07BC080916E0288606FC0CF30F4
:1029E000FCE5DF0709F480C008F082C080916E0228
:1029F000877FC8C0CE3F9CE5D90709F471C000F5B8
:102A0000C531FCE5DF0709F485C068F4C3319CE5F6
:102A1000D90709F475C008F095C00E94C5068091D9
:102A20006E028F77AFC0CC3FFCE5DF07A9F108F05D
:102A300054C0CB3FDC4509F0A7C080916F0240C075
:102A4000C230EDE5DE0709F489C058F4C1158DE503
:102A5000D80709F45AC008F069C080916F028260FB
:102A60002FC0C236EDE5DE0709F47CC0C63AFDE5AD
:102A7000DF0709F481C0C330DD4509F085C080E07F
:102A80006EC080916E0282607DC080916E0216C021
:102A900080916E02886076C080916F0282604FC024
:102AA00080916E0280626EC080916E0280646AC006
:102AB0000E94C50680916E02806864C0846062C016
:102AC00081603DC080916E028E7F5CC080916E02FD
:102AD0008D7F58C080916E0216C080916F0218C021
:102AE00080916F028D7F2BC080916E028F7E4AC0D5
:102AF00080916E028F7D46C080916E028F7B42C0B6
:102B000080916E02877F8B7F3DC080916F028D7FA9
:102B10008E7F15C080916E0282FB222720F991E002
:102B2000922790FB82F990FB83F92CC080916F0271
:102B3000982F909591708E7F892B90FB81F98093CF
:102B40006F0222C00E94C50680916E0287FB222779
:102B500020F991E0922790FB87F914C081E00E9450
:102B6000A30D12C080916E0284FB222720F991E010
:102B7000922790FB84F906C080916E02982F909561
:102B800090FB80F980936E0280916E0290916F02AB
:102B90000E941D0D0E94C50680E001C081E0DF910A
:102BA000CF910895893289F1F0F4843171F1B0F454
:102BB000873009F077C081E080930B0184E1809336
:102BC0000A018AE0809309018EE18093080188E080
:102BD0008093050188E28093040164C092EE980F0F
:102BE0009A30F0F05FC0803509F444C028F48F3487
:102BF00009F058C08AE03FC0813529F0823509F0DC
:102C000051C081E038C08FEF36C080913B028823ED
:102C100079F110923B0210923A021092390242C0AE
:102C20008D5180933B02833099F038F4813069F004
:102C30008230D9F48AE091E00DC0853099F078F0C7
:102C4000863099F484E091E005C08BE091E002C009
:102C500089E091E090933A028093390223C088E0A2
:102C600091E0F8CF85E091E0F5CF10923B021AC0D9
:102C700080E0089586EFE0913902F0913A023097B2
:102C800089F02081082E000C990B820F911D8F3F37
:102C9000910519F014F08FEF04C097FF02C0108265
:102CA00001C0808381E008950F931F9341E050E0BD
:102CB00060E070E08A019B0104C0000F111F221F19
:102CC000331F8A95D2F7C901B8010E941D071F91D1
:102CD0000F910C94C506482F50E0FA013597EF3359
:102CE000F10508F060C0EE59FF4F0C9441210E949D
:102CF000A10D55C080912802817F8E7F809328028C
:102D000081E080933C0208950E940F0248C08091A8
:102D10002802982F9095917090FB80F9809328025B
:102D200091113DC0897F877F10C08091280281FB6F
:102D3000222720F991E0922790FB81F980932802C5
:102D4000992369F18091280281608093280227C02D
:102D50008091280282FB222720F991E0922790FBA4
:102D600082F9ECCF8091280283FB222720F991E0A1
:102D7000922790FB83F9E2CF0E94C50680916E02F4
:102D800087FB222720F991E0922790FB87F9809317
:102D90006E0205C0895301C08D510E94541681E016
:102DA000089580E0FACF80E0089580E008950C94C3
:102DB000D516CF93C82F80913C02813069F038F04E
:102DC0008230C1F58C2F0E94D21581E039C00E945B
:102DD000160C823289F504C00E94160C823261F40E
:102DE0008C2F0E94D716811104C08C2F0E946B1665
:102DF0001FC081E090E01CC08C2F0E94D51681116D
:102E000016C0C43189F058F4CB3089F0C031B1F428
:102E100082E080933C0288E30E94D21508C0C93248
:102E200019F0C83321F00AC010923C0207C081E0BB
:102E3000817006C010923C0280E002C080E0F8CFB2
:102E4000CF910895CF93DF9386319C4541F5EB01F7
:102E50000E94160C982F8A81209102013091030163
:102E6000882379F09A7A81E009F480E080933D022A
:102E7000911102C069E201C065E3C9010E941819FD
:102E80000AC080913D02811102C069E201C065E380
:102E9000C9010E9423190E94580C80E001C081E002
:102EA000DF91CF9108950F931F93CF93DF93C42F9A
:102EB000D22FFC0182818823C9F0409340020E94F6
:102EC000DB1990933F0280933E0280E28C0F8830A2
:102ED00008F057C0C77081E001C0880FCA95EAF7B3
:102EE000DF91CF911F910F910C94220480914002A9
:102EF000481330C080913E0290913F020E94F31926
:102F0000883C910538F510E21D0FCD17B9F080E22D
:102F10008C0F883040F4C77081E001C0880FCA95DB
:102F2000EAF70E942904183028F581E09D2F977058
:102F300001C0880F9A95EAF70E942204802F0E9410
:102F400019041830F0F4D77081E001C0880FDA95C9
:102F5000EAF70AC080E28C0F883098F4C77081E0ED
:102F600001C0880FCA95EAF7DF91CF911F910F91A9
:102F70000C942904802FDF91CF911F910F910C9415
:102F80001904DF91CF911F910F9108950F939C0128
:102F9000CB01243F4CE5340731F188F4293DFCE5B1
:102FA0003F07D9F02A3D4CE5340779F1283D3C45EF
:102FB000A9F506E221EE41EE68ED7CE52BC0263F47
:102FC000FCE53F07E1F0A8F0273F3C4539F507E273
:102FD00025EE46EE67EF7CE51DC007E225EE45EEE7
:102FE00069ED7CE517C006E221EE40EE64EF7CE57A
:102FF00011C007E225EE44EE65EF7CE50BC006E26A
:1030000021EE42EE66EF7CE505C008E221E045EEE8
:103010006AED7CE50E94531780E008C0FC018281C4
:10302000882319F01092400201C081E00F910895A9
:103030009093850180938401089590934602809334
:1030400045020895E0914502F0914602309721F043
:103050000190F081E02D099480E00895E09145020F
:10306000F0914602309799F020911801222359F0EF
:1030700020916E0227FF07C0DC012C9111962C9342
:10308000119726E02C930280F381E02D0994089596
:10309000E0914502F0914602309739F022E0DC01E0
:1030A0002C930480F581E02D09940895209143022A
:1030B000309144022817390771F0909344028093AD
:1030C0004302E0914502F0914602309721F00680DC
:1030D000F781E02D09940895209141023091420238
:1030E0002817390771F09093420280934102E091D2
:1030F0004502F0914602309721F00084F185E02DE1
:1031000009940895FC01329680911801882331F0CA
:1031100080916E0287FF02C09EE101C096E080E0D0
:10312000915028F021912223D9F38F5FF9CF089590
:10313000662351F1209118012223E9F020916E02BB
:1031400027FF19C0462F4695469546954E31E0F427
:10315000677021E030E002C0220F331F6A95E2F76A
:10316000FC01E40FF11D828190E02823392381E0E6
:10317000232B69F409C0FC0132960896219162174D
:1031800029F0E817F907D1F780E0089581E0089564
:103190009C01FC0132969FEF80E04191461789F037
:1031A0009F3F19F4411101C0982F8F5F8630A9F716
:1031B0009F3F39F0F901E90FF11D97FDFA95628300
:1031C000089508959C012A5F3F4FFC0142814613F8
:1031D00001C01282019682179307B9F70895262F2E
:1031E0002695269526952E3168F4FC01E20FF11DF7
:1031F000677021E030E001C0220F6A95EAF7828112
:10320000282B22830895262F2695269526952E3144
:1032100070F4FC01E20FF11D677021E030E001C0A5
:10322000220F6A95EAF72095828128232283089548
:1032300020911801222329F020916E0227FD0C9481
:10324000EF180C94C81820911801222329F020911E
:103250006E0227FD0C9403190C94E21820911801BA
:10326000FC013296222331F080916E0287FF02C06A
:103270008EE101C086E0DF011D928A95E9F708958D
:1032800008950C94401983E0809347020C944119EF
:10329000811102C081E001C082E0809347020C945A
:1032A00041190C94481981E0809347020C9441190C
:1032B0000C94531908950C945A190C945B190C949E
:1032C0005A190C945A190C945A19CF930E946119E7
:1032D0000E946A110E945F19C0E08C2F0E94A21008
:1032E000811104C0CF5FC530C1F701C081E0CF912B
:1032F000089508951F920F920FB60F9211248F9385
:103300009F93AF93BF9380914802811113C0809126
:103310007A0290917B02A0917C02B0917D0241964D
:10332000A11DB11D80937A0290937B02A0937C0231
:10333000B0937D02BF91AF919F918F910F900FBE7F
:103340000F901F90189580918202843031F10E9475
:1033500070021092480220E488E190E00FB6F894E1
:10336000A895809360000FBE2093600083B7817F93
:10337000846083BF83B7816083BF7894889583B767
:103380008E7F83BF0FB6F894A89580916000886106
:1033900080936000109260000FBE08950E94C506E1
:1033A0000C94740282E084BD93E095BD9AEF97BDC2
:1033B00080936E0008952FB7F89480917A029091CF
:1033C0007B02A0917C02B0917D022FBF08952FB7A0
:1033D000F89460917A0270917B0280917C029091C6
:1033E0007D022FBF08959C014FB7F89480917A0217
:1033F00090917B02A0917C02B0917D024FBF821B15
:10340000930B089578941F920F920FB60F92112488
:103410008F939F93AF93BF9380917A0290917B0299
:10342000A0917C02B0917D020196A11DB11D8093F7
:103430007A0290937B02A0937C02B0937D02BF91AD
:10344000AF919F918F910F900FBE0F901F90189585
:1034500081E08093E00080E28093D8001092C90060
:103460008FE19EE40197F1F700C0000087E090EB48
:10347000DC0180938B0290938C02A0938D02B09319
:103480008E029CE088E10FB6F894A89580936000C6
:103490000FBE90936000FFCF80916C020895089555
:1034A00022E02093E9002FEF3091E800215035FD14
:1034B00006C035ED3A95F1F700002111F5CF2091C6
:1034C000E80025FF0BC040E050E066E070E00E949D
:1034D0008F1C8091E8008E778093E8000895CF9349
:1034E000DF9320911801222339F020916E0227FFEB
:1034F00003C060E222E002C068E021E02093E9001E
:103500002FEF3091E800215035FD06C035ED3A959A
:10351000F1F700002111F5CF2091E80025FF1DC033
:10352000EC0180911801811105C040E050E068E095
:1035300070E003C070E040E050E0CE010E948F1CBC
:103540008091E8008E778093E80080E2FE01ACE491
:10355000B2E001900D928A95E1F7DF91CF91089545
:103560008093490270934B0260934A0280918202D9
:10357000843001F582E08093E9008FEF9091E800BC
:10358000815095FD06C095ED9A95F1F700008111E7
:10359000F5CF8091E80085FF0DC040E050E063E08A
:1035A00070E089E492E00E948F1C8091E8008E77A1
:1035B0008093E8000895BC0184E00C94B01ABC012B
:1035C00083E00C94B01A80918102811109C00E949D
:1035D000201E0E947D1E8091E20084608093E200A4
:1035E00008951092810208950C94581960917E02FA
:1035F00081E0611101C080E00C9443199091820236
:1036000081E0943009F080E060917E020C944819CA
:1036100042E061EC81E00E94991D42E261EC82E0AF
:103620000E94991D9091820281E0943009F080E01F
:1036300060917E020C94511980918402833009F4C8
:1036400061C030F4813071F0823009F49AC008957D
:103650008A3009F486C08B3009F46CC0893009F0D7
:10366000A8C020C080918302813A09F0A2C0809155
:10367000E800877F8093E80080918702909188021C
:10368000892B21F460E28CE492E003C060E080E0EA
:1036900090E070E00E94DA1C8091E8008B778093C4
:1036A000E800089580918302813209F082C0809100
:1036B000870290918802029708F07BC08091E80011
:1036C000877F8093E8008091E80082FD05C08091AB
:1036D00082028111F8CF6DC02091F3008091F20039
:1036E00090E0922B029731F48091F100813011F03B
:1036F000863021F48091F10080936C028091E80083
:103700008B7753C080918302813A09F052C0809137
:10371000870290918802892B09F04BC08091E800C4
:10372000877F8093E8008091E80080FFFCCF809144
:10373000180136C0809183028132D9F580918702C9
:1037400090918802892BA9F58091E800877F80936A
:10375000E8000E94CE1D80918502809318010C9490
:10376000C50680918302813221F58091E800877F30
:103770008093E8000E94CE1D8091860280936D02A6
:10378000089580918302813AA1F48091E800877FB7
:103790008093E8008091E80080FFFCCF80916D026B
:1037A0008093F1008091E8008E778093E8000C947C
:1037B000CE1D089584B7877F84BF0FB6F894A8956F
:1037C00080916000886180936000109260000FBE5D
:1037D00090E080E80FB6F8948093610090936100C8
:1037E0000FBE0C9453190E94201E0E947D1EE2EE13
:1037F000F0E080818460808378940C9412218CE0C6
:1038000091E00C941D18809182028530A9F480917A
:103810008202853079F40E94A31980918002882366
:10382000B1F30E946519882391F30E94791C0E94CC
:10383000C506EDCF0C94CE19089508950C94201C64
:10384000292F332723303105C9F060F421303105A9
:1038500081F02230310509F044C08BE390E028EB81
:1038600031E043C021323105E1F02232310549F126
:1038700038C082E190E023EF31E037C099278130F2
:10388000910549F028F0029761F5EEE7F1E005C0F7
:10389000E4EBF1E002C0ECE8F1E0849190E09F01FC
:1038A00024C06115710541F061307105D1F489E0E2
:1038B00090E023EE31E019C089E090E02AEC31E09D
:1038C00014C06115710541F06130710551F486EB4A
:1038D00090E025E032E009C080E490E02BEB32E09C
:1038E00004C080E090E020E030E0FA0131832083E2
:1038F000089580E189BD82E189BD09B400FEFDCF54
:103900008091D8008F7D8093D8008091E000826004
:103910008093E0008091E00081FDFCCF0895CF927C
:10392000DF92EF92FF920F931F93CF93DF93EC01FF
:103930008B017A010E94ED1D811133C0E114F10465
:1039400039F0F70180819181081B190BC80FD91F2D
:10395000C12CD12C0115110519F18091E80085FDCC
:1039600016C08091E8008E778093E800E114F1049E
:1039700049F0F70180819181C80ED91ED182C082A1
:1039800085E00FC00E94ED1D882321F30AC08991B4
:103990008093F10001501109FFEFCF1ADF0ADACF4F
:1039A00080E0DF91CF911F910F91FF90EF90DF901A
:1039B000CF9008952091890230918A022617370707
:1039C00048F06115710539F42091E8002E772093B5
:1039D000E80001C0B901FC0120E06115710579F131
:1039E000809182028823F1F18530F1F18091E80025
:1039F00083FD3CC08091E80082FD2EC08091E800EC
:103A000080FFEBCF2091F3008091F20090E0922BA9
:103A10006115710551F08830910538F4219120939A
:103A2000F100615071090196F3CF21E0089709F088
:103A300020E08091E8008E778093E800CECF2111BE
:103A4000CFCF0AC080918202882361F0853061F077
:103A50008091E80083FD0AC08091E80082FFF2CFE8
:103A600080E0089582E0089583E0089581E008955C
:103A70002091890230918A022617370748F0611594
:103A8000710539F42091E8002E772093E80001C0F9
:103A9000B901FC0120E06115710591F1809182026C
:103AA000882309F440C0853009F43FC08091E800C4
:103AB00083FD3DC08091E80082FD2FC08091E80029
:103AC00080FFE9CF2091F3008091F20090E0922BEB
:103AD0006115710559F08830910540F424912093C7
:103AE000F1003196615071090196F2CF21E00897FB
:103AF00009F020E08091E8008E778093E800CBCF3A
:103B00002111CCCF0AC080918202882361F08530D8
:103B100061F08091E80083FD0AC08091E80082FF97
:103B2000F2CF80E0089582E0089583E0089581E077
:103B30000895982F973068F59093E900981739F019
:103B40007091EC002091ED005091F00003C0242F03
:103B5000762F50E021FD02C09F5FECCF3091EB004B
:103B60003E7F3093EB003091ED003D7F3093ED00D0
:103B70003091EB0031603093EB007093EC002093B8
:103B8000ED005093F0002091EE0027FDE5CF80E09E
:103B900008958F708093E90081E0089580918302F9
:103BA00087FF11C08091E80082FD05C080918202EC
:103BB0008111F8CF11C08091E8008B770BC0809104
:103BC0008202882349F08091E80080FFF8CF80913D
:103BD000E8008E778093E80008952091E40030910A
:103BE000E50095E64091EC00842F817040FF23C0F2
:103BF0008091E80080FD1DC080918202882399F0A9
:103C0000853099F08091EB0085FD11C04091E40072
:103C10005091E5002417350729F3915011F09A01CE
:103C2000E1CF84E0089582E0089583E0089581E083
:103C3000089580E008954091E80042FFDDCF0895A7
:103C40000E948E1E0E94961EE0EEF0E08081816050
:103C50008083E8EDF0E080818F77808319BCA7ED49
:103C6000B0E08C918E7F8C9380818F7E80831092C8
:103C7000810208950F931F93CF93DF930E948E1EAE
:103C80000E94961EC8EDD0E088818F778883888156
:103C90008068888388818F7D888319BC1092820216
:103CA00010927E021092800210927F0200EE10E0CD
:103CB000F80180818B7F808388818160888342E0E6
:103CC00060E080E00E94991DE1EEF0E080818E7F4F
:103CD0008083E2EEF0E08081816080838081886073
:103CE0008083F80180818E7F8083888180618883D2
:103CF000DF91CF911F910F910895E8EDF0E0808161
:103D00008F7E8083E7EDF0E080818160808384E0B6
:103D100082BF81E0809381020C943A1EE8EDF0E0CE
:103D200080818E7F80831092E20008951092DA00E5
:103D30001092E10008951F920F920FB60F92112476
:103D40002F933F934F935F936F937F938F939F93A3
:103D5000AF93BF93EF93FF938091E10082FF0BC07D
:103D60008091E20082FF07C08091E1008B7F809309
:103D7000E1000E9411218091DA0080FF1FC0809134
:103D8000D80080FF1BC08091DA008E7F8093DA001C
:103D90008091D90080FF0DC080E189BD82E189BD9D
:103DA00009B400FEFDCF81E0809382020E94E31AF5
:103DB00005C019BC109282020E94F11A8091E100A4
:103DC00080FF19C08091E20080FF15C08091E20061
:103DD0008E7F8093E2008091E20080618093E20018
:103DE0008091D80080628093D80019BC85E08093D0
:103DF00082020E94F61A8091E10084FF30C0809117
:103E0000E20084FF2CC080E189BD82E189BD09B454
:103E100000FEFDCF8091D8008F7D8093D8008091E7
:103E2000E1008F7E8093E1008091E2008F7E80939D
:103E3000E2008091E20081608093E20080917E0246
:103E4000882311F084E007C08091E30087FD02C061
:103E500081E001C083E0809382020E94FE1A80917B
:103E6000E10083FF29C08091E20083FF25C080919B
:103E7000E100877F8093E10082E0809382021092CC
:103E80007E028091E1008E7F8093E1008091E200CC
:103E90008E7F8093E2008091E20080618093E20057
:103EA00042E060E080E00E94991D8091F00088600F
:103EB0008093F0000E94F41AFF91EF91BF91AF91AF
:103EC0009F918F917F916F915F914F913F912F9132
:103ED0000F900FBE0F901F9018951F920F920FB664
:103EE0000F9211242F933F934F935F936F937F9380
:103EF0008F939F93AF93BF93CF93DF93EF93FF93F2
:103F0000C091E900CF708091EC00D82FD17080FD76
:103F1000D0E81092E9008091F000877F8093F00054
:103F200078940E94B11F1092E9008091F00088609F
:103F30008093F000CD2BCF70C093E900FF91EF91FB
:103F4000DF91CF91BF91AF919F918F917F916F91B1
:103F50005F914F913F912F910F900FBE0F901F9047
:103F600018951F93CF93DF93CDB7DEB7AA970FB6FF
:103F7000F894DEBF0FBECDBFE3E8F2E08091F10020
:103F8000819322E0EB38F207C9F70E941C1B809155
:103F9000E80083FF2EC18091830290918402492F13
:103FA00050E04A30510508F024C1FA01EF55FF4FA7
:103FB0000C944121803821F0823809F01AC108C0E0
:103FC00080917F0290918002992389F082600FC0D6
:103FD000809187028F70873008F00BC18093E900D1
:103FE0008091EB0085FB882780F91092E900909181
:103FF000E800977F9093E8008093F1001092F10021
:10400000D1C0282F2D7F09F0F4C0882319F0823009
:1040100061F0EFC080918502813009F0EAC09330F1
:1040200009F080E0809380022EC08091850281118A
:104030002AC0809187028F702FEF280F263008F05A
:10404000D8C08093E9002091EB0020FF1CC0933082
:1040500021F48091EB00806214C09091EB0090619C
:104060009093EB0021E030E0A90102C0440F551FFE
:104070008A95E2F74093EA001092EA008091EB0003
:1040800088608093EB001092E9008091E800877FC0
:104090008093E8000E94CE1DACC08111AAC010918F
:1040A00085021F778091E3008078812B8093E30065
:1040B0008091E800877F8093E8000E94CE1D809168
:1040C000E80080FFFCCF8091E30080688093E300EC
:1040D000111102C082E001C083E08093820289C096
:1040E0008058823008F085C08091850290918602C8
:1040F0008C3D53E0950779F583E08A838AE28983D2
:104100004FB7F894DE01139620E03EE051E2E32F32
:10411000F0E050935700E49120FF03C0E295EF7068
:104120003F5FEF708E2F90E0EA3010F0C79601C02D
:10413000C0968D939D932F5F243149F74FBF809197
:10414000E800877F8093E8006AE270E0CE01019684
:104150000E94DA1C16C06091870270918802AE013D
:104160004F5F5F4F0E941E1CBC01892B09F441C0A8
:104170009091E800977F9093E80089819A810E944E
:10418000381D8091E8008B778093E80032C080383A
:1041900081F58091E800877F8093E80080917E021E
:1041A0008093F1008091E8008E7772CF811121C059
:1041B000809185029091860299270297D4F480918C
:1041C000E800877F8093E8008091850280937E02DB
:1041D0000E94CE1D80917E02811106C08091E30075
:1041E00087FD02C081E001C084E0809382020E94CA
:1041F000081B8091E80083FF0AC08091E800877F58
:104200008093E8008091EB0080628093EB00AA9697
:104210000FB6F894DEBF0FBECDBFDF91CF911F91D7
:1042200008950895CF93809182028823A1F0C091D0
:10423000E900CF709091EC00892F817090FD80E8AB
:10424000C82B1092E9008091E80083FD0E94B11F05
:10425000CF70C093E900CF91089597FB072E16F415
:10426000009407D077FD09D00E94472107FC05D0B4
:104270003EF4909581959F4F0895709561957F4F7D
:104280000895EE0FFF1F0590F491E02D0994AA1BED
:10429000BB1B51E107C0AA1FBB1FA617B70710F031
:1042A000A61BB70B881F991F5A95A9F78095909563
:1042B000BC01CD010895FB01DC0104C08D9101908A
:1042C000801921F441505040C8F7881B990B08957C
:1042D000F999FECF92BD81BDF89A992780B50895CE
:1042E000A8E1B0E042E050E00C949C21262FF9991F
:1042F000FECF92BD81BDF89A019700B4021639F045
:104300001FBA20BD0FB6F894FA9AF99A0FBE089515
:104310000396272F0E9477210E947621252F0E9445
:104320007721242F0C9477210196272F0E94772143
:104330000C947621DC01CB01FC01F999FECF06C07B
:10434000F2BDE1BDF89A319600B40D924150504053
:08435000B8F70895F894FFCFBF
:10435800C800F901280850011E0A14014C1A6F1AE6
:10436800501ADF1ADB1A4F1A01E200E900EA00B519
:1043780000B600B700CD008301CC008A01920194F9
:10438800012102230224022502260227022A02B35F
:1043980000B4006F007000818283E200E900EA0047
:1043A800B500B600B700CD008301CC008A019201A8
:1043B80094012102230224022502260227022A024E
:1043C800B300B4006F007000818283F43397359492
:0443D8006636C6344B
:00000001FF
